:100000008AEF0EF0FFFF200000C016F001C015F0CF
:10001000E1CF17F0E2CF18F09DAA74D09EAA72D05B
:10002000AECFF8F0ABA20FD0AB98AECFF8F0AB8864
:10003000010E04011925006E000E1A21016E00C088
:1000400019F401C01AF4ABA40FD00401AB9EAB8E1F
:10005000010E1925006E000E1A21016E00C019F460
:1000600001C01AF4AECFF8F00001F8510D0A08E013
:100070000401AA51000802E1A9517E0801E327D03A
:10008000010E0001FD6F000EFE6F0401AA51000871
:1000900002E1A9517E0805E2020E0001FD6F000E8B
:1000A000FE6F9D9A990E0401A925E16E030EAA2107
:1000B000E26EE1CFE1FFE2CFE2FFE66AA9C493F38B
:1000C000AAC494F3A96BAA6B0001F86B1BD0990E1C
:1000D0000401A925E16E030EAA21E26EE1CFE1FF42
:1000E000E2CFE2FFF8C0E6FFA9C493F3AAC494F3F9
:1000F000010EA925006E000EAA21016E00C0A9F410
:1001000001C0AAF49DA01FD09EA01DD0010E010128
:10011000015D006E000E0259016E00C001F101C0C8
:1001200002F1000E025D02E1010E015D07E29D9009
:10013000CD90010E0001EE6F000EEF6F3C0ECF6E02
:10014000B00ECE6E9E9016C000F015C001F017C024
:10015000E1FF18C0E2FF110072B201D0FDD7DBC48D
:1001600073FF1200ACB202D00000FCD7DBC4ADFFBD
:100170001200F250026EF29E0500FF6A0150FE6E00
:100180000050FD6E02BEF28E1200C7B409D01F0EE1
:10019000C514016E0150000A03E1010E006E01D08A
:1001A000006A1200C58412009E96D5C4C9FFA5C07E
:1001B000D6F4A6C0D7F4A7C0D8F4A8C0D9F4C7A471
:1001C00022D00001A551A611A711A8111BE004011E
:1001D000D651D711D811D9110EE1F6C0E1FFF7C001
:1001E000E2FF040EE66EF4C000F0F5C001F0C1DFDE
:1001F000010E006E3BD0010E0401D65F000ED75BEE
:10020000D85BD95BDCD7A5C0D6F4A6C0D7F4A7C00D
:10021000D8F4A8C0D9F49EB622D00001A551A611E9
:10022000A711A8111BE00401D651D711D811D9117B
:100230000EE1F6C0E1FFF7C0E2FF040EE66EF4C087
:1002400000F0F5C001F095DF010E006E0FD0010E39
:100250000401D65F000ED75BD85BD95BDCD7C5BC89
:1002600002D0006A03D0C584020E006E1200A5C041
:10027000D7F4A6C0D8F4A7C0D9F4A8C0DAF4040112
:10028000D56BD66BD651120802E1D5518E0808E322
:100290007CDF005201E004D00401D54BD62BF2D70D
:1002A0000401120ED65D02E18F0ED55D03E37B0ED5
:1002B000006E26D0C580C5A022D00001A551A61190
:1002C000A711A8111BE00401D751D811D911DA11D7
:1002D0000EE1F6C0E1FFF7C0E2FF050EE66EF4C0E6
:1002E00000F0F5C001F045DF010E006E09D0010EEF
:1002F0000401D75F000ED85BD95BDA5BDCD7006AFC
:100300001200086A080E0C6E003408360450085EAD
:10031000D8B002D00826D89000360C2EF5D712009F
:100320000B6A0A6A096A00500402F4CF09F0F3CF9D
:1003300008F001500502F4CF0BF0F3CF0AF00050A3
:100340000502F3500926F4500A22E86A0B220150F4
:100350000402F3500926F4500A22E86A0B2208C06E
:1003600000F009C001F00AC002F00BC003F0120057
:100370007EDF780E0401D56F17DF07DF0050000A1B
:1003800001E1FBD7800E0401D56F0EDFFEDE0050C9
:10039000000A01E1FBD7D2C4D5F406DFF6DE005037
:1003A000000A01E1FBD7FEDE1200013408360936EF
:1003B0000450085E0550D8A0053C095E00360136A1
:1003C0000F0E0C6E013408360936045000A006D01A
:1003D000085E0550D8A0053C095E05D008260550EA
:1003E000D8B0053C0926003601360C2EEBD700B0FC
:1003F00006D0045008260550D8B0053C0926000058
:100400001200800E0401D319006E800E005C02E120
:10041000000ED25D08E2D2510008006ED3C401F094
:10042000000E015604D0D2C400F0D3C401F0120073
:10043000030E006ED3C407F0000E086E005004E0F7
:100440000732079EFF0FFBD7000E086E070E040150
:10045000D315096E0A6A000E0A16000E0A6E070E00
:10046000026E07C000F008C001F0025005E000363F
:1004700000900136FF0FFAD70401D2510026000E7A
:10048000012200C003F001C004F08B0E0024E96ECD
:10049000010E0120EA6EE9CFE9FFEACFEAFFEECFD5
:1004A00005F0000E066E000E066ED451010A12E130
:1004B00009C002F0010E006E000E016E025005E050
:1004C000003600900136FF0FFAD700500512015098
:1004D000061213D009C002F0010E006E000E016E6C
:1004E000025005E0003600900136FF0FFAD7001EDB
:1004F000011E00500516015006168B0E0324E16EF6
:10050000010E0420E26EE1CFE1FFE2CFE2FF05C081
:10051000E6FF1200ACDE780E0401D56F45DE35DE55
:100520000050000A01E1FBD7400E0401D56F3CDE0C
:100530002CDE0050000A01E1FBD7D2C4D5F434DE32
:1005400024DE0050000A01E1FBD72CDE1200300E41
:10055000CD6E3C0ECF6EB00ECE6EBDC401F1BEC4EA
:1005600002F10001EE6BEF6BCD809E909D8012003A
:10057000220E0C6E086A096A0A6A0B6A0C06D8B465
:100580001FD0D8900B320A320932083203320232BD
:1005900001320032D8A0F2D70C06D8B409D00450EA
:1005A00008260550092206500A2207500B22EAD7D6
:1005B000045008260550092206500A2207500B2233
:1005C00012000401BD51BF5DD26F000EBFBFFF0E10
:1005D000D36F000EBDBFFF0ED35B13DF00C0CAF4A4
:1005E00001C0CBF4BE51C05DD26F000EC0BFFF0E84
:1005F000D36F000EBEBFFF0ED35B03DF00C0CCF491
:1006000001C0CDF4BDC4C2F4000EBDBFFF0EC36F68
:10061000BEC4C4F4000EBEBFFF0EC56F800EBF196E
:10062000006E800EBD19005C05E2FF0EC66FFF0E66
:10063000C76F04D0010EC66F000EC76F800EC019C1
:10064000006E800EBE19005C05E2FF0EC86FFF0E43
:10065000C96F04D0010EC86F000EC96F800ECB1990
:10066000006E800ECD19005C02E1CC51CA5D5AE3E8
:10067000CCC4CEF4CDC4CFF4CE37CE91CF37CA514F
:10068000CE5FCB51CF5BD06BD16B800ECB19006EA0
:10069000800ED119005C02E1D051CA5D42E3C2C4B0
:1006A000D2F4C4C4D3F4C1C4D4F4C2DE800E0401B5
:1006B000CF19006E800E005C02E1000ECE5D10E2EC
:1006C000CCC400F0CDC401F00036009001360050DB
:1006D000CE270150CF23C651C227C751C3231ED0F6
:1006E000CCC400F0CDC401F00036009001360050BB
:1006F000CE270150CF23CAC400F0CBC401F000368E
:10070000009001360050CE5F0150CF5BC651C2272A
:10071000C751C323C851C427C951C523D04BD12BBE
:10072000B4D759D0CAC4CEF4CBC4CFF4CE37CE910F
:10073000CF37CC51CE5FCD51CF5BD06BD16B800E1C
:10074000CD19006E800ED119005C02E1D051CC5D54
:1007500042E3C2C4D2F4C4C4D3F4C1C4D4F468DE46
:10076000800E0401CF19006E800E005C02E1000EC5
:10077000CE5D10E2CAC400F0CBC401F00036009098
:1007800001360050CE270150CF23C851C427C9518C
:10079000C5231ED0CAC400F0CBC401F000360090BF
:1007A00001360050CE270150CF23CCC400F0CDC479
:1007B00001F00036009001360050CE5F0150CF5B53
:1007C000C651C227C751C323C851C427C951C52325
:1007D000D04BD12BB4D71200BDC404F0BEC405F079
:1007E00004C0E9FF05C0EAFFEE5203E0044A052A0F
:1007F000F7D704C002F005C003F0044A052ABFC4BD
:1008000000F0C0C401F00401BF4BC02B00C0E9FFE1
:1008100001C0EAFF02C0E1FF03C0E2FFEECFE6FF46
:1008200002C0E9FF03C0EAFFEE5201E0E2D7BDC417
:1008300000F0BEC401F01200BFC4F6FFC0C4F7FF51
:10084000C1C4F8FF0900F5CF00F0005218E0BFC4A2
:10085000F6FFC0C4F7FFC1C4F8FF0900F5CF00F0F0
:10086000BDC4E1FFBEC4E2FF00C0E6FF0401BD4B12
:10087000BE2B010EBF27000EC023C123DDD7BDC490
:10088000E1FFBEC4E2FFE66A1200BDC4F6FFBEC4CB
:10089000F7FFBFC4F8FF0900F5CF00F0005211E0E8
:1008A000BDC4F6FFBEC4F7FFBFC4F8FF0900F5CF13
:1008B000DBF458DC010E0401BD27000EBE23BF236C
:1008C000E4D7060E0D6E0D2EFED7000012000401B7
:1008D000C06BBDC4E9FFBEC4EAFFEECFBFF4BF5199
:1008E000000A0EE0BFC4DBF43DDC0401C02BC051A4
:1008F000BD25E96E000EBE21EA6EEECFBFF4EFD744
:100900001200200E0401D26F33DD0401D26B30DD02
:10091000210E0401D26F2CDDBDC4D2F429DD040107
:10092000BD510F0FD26F24DD220E0401D26F20DDE6
:10093000010E0401D26F1CDD030E0401D26F18DD1D
:100940000401BF6BC06B800EC019006E800E005C8E
:1009500002E1300EBF5D2CE2030E006E000E016E50
:10096000BEC404F0000E056EDBDCA90E0024E96EA7
:10097000000E0120EA6EE9CFE9FFEACFEAFFBF519E
:10098000EE24F66EC051EE20F76E000EC0BFFF0ED3
:10099000EE20F86EF6CFF6FFF7CFF7FFF8CFF8FFAF
:1009A0000900F5CFD2F4B6DD0401BF4BC02BCBD785
:1009B00012000D0E0401DB6FB2EC00F00A0E040110
:1009C000DB6FB2EC00F012000450000A08E10550A1
:1009D000000A05E1FF0E006E7F0E016E57D00D6A12
:1009E000096A086A01500010D8B4000C01500518BB
:1009F0000A6E0ABE0D1E0B6A05AE05D0041E051E4A
:100A0000042AD8B4052A01AE05D0001E011E002A12
:100A1000D8B4012A015005100A6E0ABE10D0C5DCF8
:100A20000BB020D00DAE000C001E011E002AD8B461
:100A3000012A081E091E082AD8B4092A000C05AE8E
:100A40000DD001BE07D00150096E0050086E016A3A
:100A5000006AE8D7016A006A002A000C011E001E25
:100A60000B2ADDD7082AD8B4092A0450085CD8A478
:100A7000D9D70550095CD8A4D5D7096A086A002AD5
:100A8000D8B4012A01AECED70000FF0C120003013A
:100A9000936B946B000E945D02E17F0E935D16E202
:100AA000990E9325E16E030E9421E26EE1CFE1FFF2
:100AB000E2CFE2FFE66A010E9325006E000E94215C
:100AC000016E00C093F301C094F3E4D70401A96B55
:100AD000AA6B0301936B946B0001F86BFD6BFE6BCB
:100AE000AB98AB88F28CAECFF8F09D8A1200BDC4F3
:100AF00002F0BEC403F002C000F003C001F0024ADD
:100B0000032A00C0E9FF01C0EAFFEE5201E0F3D77B
:100B10000401BD51025C006EBE510358016E010E0E
:100B2000005E000E015A12000401C06B030EC05D8E
:100B30000AE2C051BE25E16E000EBF21E26E200E1A
:100B4000E66EC02BF3D7C051BE25E16E000EBF216B
:100B5000E26EE66AC007C051BE25C16F000EBF211C
:100B6000C26F0A0E046EBDC400F081EC01F008C033
:100B700000F0300E0026C1C4E1FFC2C4E2FF00C095
:100B8000E6FF0A0E046EBDC400F081EC01F000C067
:100B9000BDF40050000A01E102D0C007DCD712000A
:100BA0000401BE51B00FD26FB8EC01F00F0E04017A
:100BB000BD15D26FB8EC01F0F00E0401BD15D26F77
:100BC000D233D29FD233D29FD233D29FD233D29F4D
:100BD000D289B8EC01F01200640E0001F96F010E29
:100BE000FA6FDB0EFB6F040EFC6FFF0E04019D6FAE
:100BF000FF0E9E6F000E9F6F000EA06FFF0EA16F85
:100C0000FF0EA26F000EA36F000EA46FFF0EA56F64
:100C1000FF0EA66F000EA76F000EA86FAC8A900E95
:100C2000AB6E948E949C9EAA03D0AECF00F0FBD7FF
:100C30001200826A0F013A6B948E949C94928B926C
:100C40003F0E806E386BEF0E926E546BFF0E816E0E
:100C5000830E936E396B606A12008A0E0101036F76
:100C6000010E046F000E056F000E066F6E0E076F0B
:100C7000020E086F000E096F000E0A6FFF0E0301CF
:100C80008B6FFF0E8C6F000E8D6F000E8E6FFF0E40
:100C90008F6FFF0E906FFF0E916FFF0E926FA80E79
:100CA0000001F06F010EF16FD50EF26F040EF36FBD
:100CB000A40E0401AB6F010EAC6F000EAD6F000E01
:100CC000AE6F949894968B988B9694889486C79ED2
:100CD000C79C380EC66E12000900F5CFE6FF00066D
:100CE000FBE10106F9E112008978800E030A006E2B
:100CF000800E0401B019005C02E1AF51E70804E284
:100D0000E70EAF6F030EB06FAFC4B9F4B0C4BAF45E
:100D1000BEDEAFC4BDF4B0C4BEF419DC4E0E040197
:100D2000BD6F440EBE6F000EBF6FAFDD640E046E6C
:100D3000000E056EB9C400F0BAC401F045DE800EA5
:100D4000026E800E0118025C02E1005000080EE203
:100D5000640E046E000E056EB9C400F0BAC401F052
:100D600033DE300E002600C0B1F403D0200E0401A3
:100D7000B16F640E046E000E056EB9C400F0BAC403
:100D800001F022DE08C000F009C001F000C0B9F493
:100D900001C0BAF40A0E046E000E056E15DE800E58
:100DA000026E800E0118025C02E1005000080EE2A3
:100DB0000A0E046E000E056EB9C400F0BAC401F04C
:100DC00003DE300E00240401B26F03D00401300EA4
:100DD000B26F2C0EB36F0A0E046E000E056EB9C40E
:100DE00000F0BAC401F0F0DD08C000F009C001F065
:100DF000300E00240401B46FB56BB10EBD6F040E4C
:100E0000BE6F65DD370EBD6F470EBE6F000EBF6F44
:100E10003CDD000E0001FE1902E1000EFD1907E1A4
:100E2000000EEF1902E1000EEE1901E1F2D7EE6BB0
:100E3000EF6BFD6BFE6BBDDD1200210ECD6ECD8222
:100E40003C0ECF6EB00ECE6E9E909F800101016B66
:100E5000026B0001EE6BEF6BCD909D901200AE0E19
:100E60000401D26FB8EC01F0050E0B6E0F0E0C6E84
:100E7000F10E0D6E0D2EFED70C2EFCD70B2EFAD7D1
:100E8000AF0E0401D26FB8EC01F0030E0B6E080E2A
:100E90000C6E770E0D6E0D2EFED70C2EFCD70B2E82
:100EA000FAD7B00E0401D26FB8EC01F00401D26B96
:100EB000B8EC01F0030E0401D26FB8EC01F0200E83
:100EC0000401D26FB8EC01F0020E0401D26FB8EC4D
:100ED00001F0210E0401D26FB8EC01F00401D26BD5
:100EE000B8EC01F07F0E0401D26FB8EC01F0220ED5
:100EF0000401D26FB8EC01F00401D26BB8EC01F040
:100F0000030E0401D26FB8EC01F0A10E0401D26F00
:100F1000B8EC01F0A40E0401D26FB8EC01F0A60EFB
:100F20000401D26FB8EC01F0C80E0401D26FB8EC26
:100F300001F0D30E0401D26FB8EC01F03F0E0401B2
:100F4000D26FB8EC01F0D50E0401D26FB8EC01F00D
:100F5000800E0401D26FB8EC01F0A80E0401D26F2C
:100F6000B8EC01F03F0E0401D26FB8EC01F0D60EE0
:100F70000401D26FB8EC01F0800E0401D26FB8EC1E
:100F800001F0D90E0401D26FB8EC01F01F0E04017C
:100F9000D26FB8EC01F0DA0E0401D26FB8EC01F0B8
:100FA000200E0401D26FB8EC01F0EE0E0401D26FF6
:100FB000B8EC01F0810E0401D26FB8EC01F07F0EA5
:100FC0000401D26FB8EC01F02E0E0401D26FB8EC20
:100FD00001F0DB0E0401D26FB8EC01F0400E040109
:100FE000D26FB8EC01F08D0E0401D26FB8EC01F0B5
:100FF000140E0401D26FB8EC01F0AF0E0401D26FF1
:10100000B8EC01F012000401BD6BBE6BC9DD040138
:10101000AF6B040EAF5D25E2AF51B00FD26FB8ECED
:1010200001F0420E0D6E0D2EFED700000401D26BB2
:10103000B8EC01F0100E0401D26FB8EC01F004011D
:10104000B06B800EB05D0BE200C1D2F48AEC02F00E
:101050000D0E0D6E0D2EFED70401B02BF2D7AF2B67
:10106000D8D712000101006B0401B86BB96BBA6BE1
:10107000BB6BBC6BAFC4BBF4B0C4BCF4AFC4BDF4B9
:10108000B0C4BEF48DDDAAD10401B951B125E96E19
:10109000000EB221EA6EE9CFE9FFEACFEAFFEE5097
:1010A000000AD8B476D0040EBC5D73E2B951B12504
:1010B000E96E000EB221EA6EE9CFE9FFEACFEAFF5E
:1010C000200EEE5C0101006F0401BB51780808E2BC
:1010D000AFC4BBF4BC2BAFC4BDF4BCC4BEF460DD74
:1010E0000401B86B060EB85D50E2060E006E000EED
:1010F000016E026E036E00C104F0000E056E066EF6
:10110000076EB8EC02F0380E0026330E0122000EF6
:101110000222B8510024F66E000E0120F76E000E78
:101120000220F86EF6CFF6FFF7CFF7FFF8CFF8FF03
:101130000900F5CF00F000C0BAF400C0D2F48AEC88
:1011400002F0070E026EBCC400F0000E016E0250E9
:1011500005E0003600900136FF0FFAD70401BB51BD
:101160000026000E0122B8510026000E01228B0E2F
:101170000024E16E010E0120E26EE1CFE1FFE2CF3B
:10118000E2FFBAC4E6FFB82BADD7060EBB27B92BDA
:101190007BD7D26B8AEC02F00401D26B8AEC02F0AE
:1011A0002BD1B1C4BDF4B2C4BEF4A1DC00C0B4F410
:1011B00001C0B5F4B96BB951B125E96E000EB22189
:1011C000EA6EE9CFE9FFEACFEAFFEE50000AD8B4B1
:1011D00085D0100EB95DD8B081D0B951B125E96E76
:1011E000000EB221EA6EE9CFE9FFEACFEAFF200E56
:1011F000EE5C0101006FBBC4BDF4BCC4BEF4D0DC26
:101200000401B86B080EB85D2BE2040E026E00C13B
:1012100000F0000E016E025005E00036009001362D
:10122000FF0FFAD7B8510026000E0122480E002405
:10123000F66E2D0E0120F76E000EF86E000E01BE48
:10124000FF0EF822F6CFF6FFF7CFF7FFF8CFF8FF43
:101250000900F5CFD2F48AEC02F00401B82BD2D702
:10126000BBC4BDF4BC51010FBE6F9ADC0401B86B66
:10127000080EB85D2FE2040E026E00C100F0000EF1
:10128000016E025005E0003600900136FF0FFAD7DC
:10129000B8510026000E0122080E0026000E012281
:1012A000480E0024F66E2D0E0120F76E000EF86E2B
:1012B000000E01BEFF0EF822F6CFF6FFF7CFF7FFC4
:1012C000F8CFF8FF0900F5CFD2F48AEC02F0040160
:1012D000B82BCED7080EBB27B92B6DD78DD0B1C494
:1012E000BDF4B2C4BEF403DC00C0B6F401C0B7F470
:1012F000800E026E800E0118025C02E100500008B0
:10130000D8B06AD0B86B800E006E800EB719005C42
:1013100002E1B651B85D60E2070EB825B46FB56B57
:10132000000EB523B651B45FB751B55B040E006E25
:10133000005005E0B437B491B537FF0FFAD7B85174
:10134000B125E96E000EB221EA6EE9CFE9FFEACFDE
:10135000EAFFEECF01F001C000F101502F080DE2CD
:101360003A0E0101005D09E2B4C4BDF4300E005D27
:101370000401BE6F81EC04F02CD020D00401B4C471
:10138000BDF40A0EBE6F81EC04F023D00401B4C496
:10139000BDF40B0EBE6F81EC04F01BD00401B4C48D
:1013A000BDF40C0EBE6F81EC04F013D00401B4C484
:1013B000BDF40B0EBE6F81EC04F00BD001010051A7
:1013C0002E0ADCE00051200AE1E00051B00AE6E01C
:1013D000EDD70401B82B97D70FD00ED00401B3512D
:1013E000010AD8B451D6B351020AD8B4DAD6B351EF
:1013F000030AD8B474D7F1D712008B8237EC01F00E
:101400008B9200008B8200C1D5F4D4EC00F0005028
:10141000000A08E02E0E0401DB6FB2EC00F00401BC
:10142000AF6B40D0040195C3BDF496C3BEF4ED0E7E
:10143000BF6F450EC06F000EC16F1CEC04F095C36A
:10144000BDF496C3BEF477EC05F000C09BF401C078
:101450009CF400C1BDF40B0EBE6F010EBF6F94EC87
:1014600005F09B51030195250401BD6F9C510301BB
:1014700096210401BE6F0B0EBF6F010EC06FECEC26
:1014800003F095C3BDF496C3BEF467EC04F02B0ED5
:10149000BD6F470EBE6F000EBF6F45EC04F0010E2E
:1014A0000401AF6FD2EC00F08B92AFC400F01200D9
:1014B000200E0401D26FB8EC01F00401D26BB8EC3D
:1014C00001F0210E0401D26FB8EC01F0AFC4D2F4E8
:1014D000B8EC01F00401AF51070FD26FB8EC01F086
:1014E000220E0401D26FB8EC01F0B0C4D2F4B8EC13
:1014F00001F00401B051010FD26FB8EC01F004010A
:10150000B26BB36B800EB319006E800E005C02E10B
:10151000070EB25D2EE2030E006E000E016EB1C426
:1015200004F0000E056E90EC01F0190E0024E96E37
:10153000000E0120EA6EE9CFE9FFEACFEAFFB251DF
:10154000EE24F66EB351EE20F76E000EB3BFFF0E21
:10155000EE20F86EF6CFF6FFF7CFF7FFF8CFF8FFE3
:101560000900F5CFD2F48AEC02F00401B24BB32BA0
:10157000C9D71200AFC4BDF4B0C4BEF4D0EC05F0BE
:10158000200E0401B15DD8A048D137EC01F0780EEF
:101590000401D56FD4EC00F0C5EC00F00050000A57
:1015A00001E1FAD7400E0401D56FD4EC00F0C5EC90
:1015B00000F00050000A01E1FAD70401B151B00A6D
:1015C00005E0200EB15D0101006F03D001015C0E4A
:1015D000006F060E006E000E016E026E036E00C1FB
:1015E00004F0000E056E066E076EB8EC02F0380EC1
:1015F0000024F66E330E0120F76E000E0220F86E06
:10160000F6CFF6FFF7CFF7FFF8CFF8FF0900F5CFD9
:10161000D5F4D4EC00F0C5EC00F00050000A01E174
:10162000FAD7060E006E000E016E026E036E00C148
:1016300004F0000E056E066E076EB8EC02F0380E70
:101640000026330E0122000E0222010E0024F66E47
:10165000000E0120F76E000E0220F86EF6CFF6FFA6
:10166000F7CFF7FFF8CFF8FF0900F5CFD5F4D4ECAA
:1016700000F0C5EC00F00050000A01E1FAD7060EB8
:10168000006E000E016E026E036E00C104F0000ECB
:10169000056E066E076EB8EC02F0380E0026330EAB
:1016A0000122000E0222020E0024F66E000E01201E
:1016B000F76E000E0220F86EF6CFF6FFF7CFF7FFB9
:1016C000F8CFF8FF0900F5CFD5F4D4EC00F0C5EC65
:1016D00000F00050000A01E1FAD7060E006E000E7D
:1016E000016E026E036E00C104F0000E056E066E00
:1016F000076EB8EC02F0380E0026330E0122000E01
:101700000222030E0024F66E000E0120F76E000E7A
:101710000220F86EF6CFF6FFF7CFF7FFF8CFF8FF0D
:101720000900F5CFD5F4D4EC00F0C5EC00F0005082
:10173000000A01E1FAD7060E006E000E016E026E7D
:10174000036E00C104F0000E056E066E076EB8EC65
:1017500002F0380E0026330E0122000E0222040E83
:101760000024F66E000E0120F76E000E0220F86EC7
:10177000F6CFF6FFF7CFF7FFF8CFF8FF0900F5CF68
:10178000D5F4D4EC00F0C5EC00F00050000A01E103
:10179000FAD7060E006E000E016E026E036E00C1D7
:1017A00004F0000E056E066E076EB8EC02F0380EFF
:1017B0000026330E0122000E0222050E0024F66ED2
:1017C000000E0120F76E000E0220F86EF6CFF6FF35
:1017D000F7CFF7FFF8CFF8FF0900F5CFD5F4D4EC39
:1017E00000F0C5EC00F00050000A01E1FAD7040156
:1017F000D56BD4EC00F0C5EC00F00050000A01E11C
:10180000FAD70401D56BD4EC00F0C5EC00F0005021
:10181000000A01E1FAD7D2EC00F01200210E040117
:10182000D26FB8EC01F00401D26BB8EC01F07F0E7E
:101830000401D26FB8EC01F0220E0401D26FB8ECB3
:1018400001F00401D26BB8EC01F0030E0401D26F79
:10185000B8EC01F0D30E0401D26FB8EC01F0400EE9
:101860000401D26FB8EC01F00401BD6BBE6BD0EC8B
:1018700005F00101006B040E005D26E20051B00F7F
:101880000401D26FB8EC01F0010E0401D26FB8EC84
:1018900001F0100E0401D26FB8EC01F00D0E0D6EC8
:1018A0000D2EFED70401AF6B800EAF5D0AE2D26B46
:1018B0008AEC02F00D0E0D6E0D2EFED70401AF2B3B
:1018C000F3D70101002BD7D72E0E0401D26FB8EC4D
:1018D00001F00401BD6BBE6BD0EC05F01200016A93
:1018E000026A800E0218006E800E020A005C02E19D
:1018F000000E015C0EE28B0E0124E16E010E02204F
:10190000E26EE1CFE1FFE2CFE2FFE66A014A022A9E
:10191000E8D712000101006B0401B56BB66BB76B21
:10192000B86BB351000A31E0B151AF5D05E2AFC40D
:10193000B5F4B1C4B6F404D0B1C4B5F4AFC4B6F4D0
:10194000B251B05D05E2B0C4B7F4B2C4B8F404D08B
:10195000B2C4B7F4B0C4B8F4B551B65D15E3B7C4BA
:1019600000F1010100510401B85D0BE3B5C4D2F4EC
:1019700000C1D3F4B4C4D4F418EC02F00101002B7C
:10198000F0D70401B52BE8D730D0AFC4BDF4B0C454
:10199000BEF4B1C4BFF4B0C4C0F4B4C4C1F4E1EC4B
:1019A00002F0AFC4BDF4B2C4BEF4B1C4BFF4B2C45B
:1019B000C0F4B4C4C1F4E1EC02F0AFC4BDF4B0C4EF
:1019C000BEF4AFC4BFF4B2C4C0F4B4C4C1F4E1EC1B
:1019D00002F0B1C4BDF4B0C4BEF4B1C4BFF4B2C42B
:1019E000C0F4B4C4C1F4E1EC02F012000401BD6B18
:1019F000BE6BD0EC05F00101006B040E005D39E216
:101A00000051B00F0401D26FB8EC01F0850E0D6EDD
:101A10000D2EFED70401AF6B800EAF5D27E2070EDF
:101A2000026E00C100F0000E016E025005E00036AB
:101A300000900136FF0FFAD7AF510026000E0122A9
:101A40008B0E0024E96E010E0120EA6EE9CFE9FF5A
:101A5000EACFEAFFEECFD2F48AEC02F01A0E0D6E56
:101A60000D2EFED700000401AF2BD6D70101002BAD
:101A7000C4D70401BD6BBE6BD0EC05F012008D0E17
:101A80000401D26FB8EC01F0140E0401D26FB8EC6F
:101A900001F0AF0E0401D26FB8EC01F012000401A6
:101AA000B46BB56BB66BB76BB86BB96BB1C4B6F44E
:101AB000000EB76FB6510108B86FB7C4B9F4000E85
:101AC000B957B251000A45E0B451AF5DBD6FB65190
:101AD000B025006E00C0BEF4B451AF25BF6F00C08A
:101AE000C0F4B3C4C1F4E1EC02F0B451AF5DBD6F1A
:101AF000B651B05D006E00C0BEF4B451AF25BF6FEB
:101B000000C0C0F4B3C4C1F4E1EC02F0B651AF5D63
:101B1000BD6FB451B025006E00C0BEF4B651AF2504
:101B2000BF6F00C0C0F4B3C4C1F4E1EC02F0B65121
:101B3000AF5DBD6FB451B05D006E00C0BEF4B65174
:101B4000AF25BF6F00C0C0F4B3C4C1F4E1EC02F034
:101B500057D0B451AF25D26FB651B025D36FB3C4AF
:101B6000D4F418EC02F00401B651AF25D26FB45191
:101B7000B025D36FB3C4D4F418EC02F00401B4510F
:101B8000AF5DD26FB651B025D36FB3C4D4F418ECA7
:101B900002F00401B651AF5DD26FB451B025D36FDE
:101BA000B3C4D4F418EC02F00401B651AF25D26FDF
:101BB000B451B05DD36FB3C4D4F418EC02F0040197
:101BC000B451AF25D26FB651B05DD36FB3C4D4F466
:101BD00018EC02F00401B451AF5DD26FB651B05DA4
:101BE000D36FB3C4D4F418EC02F00401B651AF5D66
:101BF000D26FB451B05DD36FB3C4D4F418EC02F01B
:101C0000800E0401B919006E800E005C02E1000E26
:101C1000B85D12E2B4C400F0B5C401F00036009023
:101C20000136030E0026000E01220050B827015095
:101C3000B923B44BB52B1BD0B651B45D036EB7516D
:101C4000B559046E03C000F004C001F000360090E6
:101C50000136050E0026000E01220050B827015063
:101C6000B923B44BB52B010EB65F000EB75B800EE7
:101C7000B719006E800EB519005C02E1B451B65D73
:101C8000D8B01FD712000401B76BB86B030EB215A2
:101C9000016E0150000A07E1B2C4B6F4B633B69F34
:101CA000B633B69F07D0B2C4B6F4B633B69FB633D8
:101CB000B69FB62BB0C4B6F4B251B65D2AE2AFC43B
:101CC000BDF4B6C4BEF4D0EC05F0AFC400F104011D
:101CD000B1510101005D1AE20401B751B325F66E5E
:101CE000B851B421F76E000EB521F86EF6CFF6FFAD
:101CF000F7CFF7FFF8CFF8FF0900F5CFD2F4B74BD5
:101D0000B82B8AEC02F00101002BE1D70401B62BBD
:101D1000D3D71200CCEC23F09B6A720ED36ED26A3A
:101D2000030E0B6E080E0C6E770E0D6E0D2EFED789
:101D30000C2EFCD70B2EFAD719EC06F00301976B8B
:101D4000986B800E9819006E800E020A005C02E10A
:101D5000000E975D0EE28B0E9725E16E010E982125
:101D6000E26EE1CFE1FFE2CFE2FFE66A974B982B0C
:101D7000E8D7976B986B800E9819006E800E005C08
:101D800002E1020E975D1DE28998050E0B6E0F0EA3
:101D90000C6EF10E0D6E0D2EFED70C2EFCD70B2EF9
:101DA000FAD78988050E0B6E0F0E0C6EF10E0D6EB4
:101DB0000D2EFED70C2EFCD70B2EFAD7974B982B57
:101DC000DAD71B0E956F040E966FB886B06A220E96
:101DD000AF6EAC84ECEC05F0030E0B6E080E0C6ECF
:101DE000770E0D6E0D2EFED70C2EFCD70B2EFAD7CC
:101DF000D9EC04F0A00E0401BD6F460EBE6F000EBC
:101E0000BF6F45EC04F00301976B986B800E981937
:101E1000006E800E005C02E1090E975D20E2030E69
:101E2000006E000E016E97C304F098C305F090ECAD
:101E300001F0D00E0024E96E000E0120EA6EE9CF19
:101E4000E9FFEACFEAFFEECFBDF4EECFBEF4EECF6E
:101E5000BFF445EC04F00301974B982BD7D7150E30
:101E60000B6E4B0E0C6EBE0E0D6E0D2EFED70C2E95
:101E7000FCD70B2EFAD70000D9EC04F0920E040127
:101E8000BD6F470EBE6F000EBF6F45EC04F0060E2F
:101E90000401BD6F440EBE6F000EBF6F45EC04F031
:101EA000D08E9F8A9E8AAB88F28CF28E04019B6B47
:101EB0009C6BE60EBD6F400EBE6F000EBF6F45EC13
:101EC00004F01DEC07F0140E0401BD6F000EBE6F90
:101ED000A7EC02F0240EAD6ED9EC04F0000E000168
:101EE000EF1902E1000EEE1901E1F8D7230EAD6EF5
:101EF000D9EC04F004019B6B9C6BF29E110EBD6F3C
:101F0000470EBE6F000EBF6F45EC04F0280EC86E82
:101F10002DEC06F00B0E0B6E260E0C6E5D0E0D6E8C
:101F20000D2EFED70C2EFCD70B2EFAD7000000008A
:101F3000200E0301976F000E986F800E9819006EA7
:101F4000800E005C02E1FE0E975D18E297C300F17F
:101F5000FDEC09F000C0FFF0030E0B6E080E0C6ED6
:101F6000770E0D6E0D2EFED70C2EFCD70B2EFAD74A
:101F7000020E03019727000E9823DFD7D2EC00F062
:101F8000D9EC04F07D0E0401BD6F400EBE6F000E53
:101F9000BF6F45EC04F02FEC07F00B0E0B6E260E16
:101FA0000C6E5D0E0D6E0D2EFED70C2EFCD70B2E7B
:101FB000FAD70000000063DD19DD1E0E0401BD6FBD
:101FC000470EBE6F000EBF6F45EC04F027DCF28EAB
:101FD000C20E0401BD6F3E0EBE6F000EBF6F45EC1A
:101FE00004F0FF0E0101006F03EC08F0140EAF6F58
:101FF000000EB06F74EC06F08B0E0401BD6F3F0E47
:10200000BE6F000EBF6F45EC04F00101006B03ECE6
:1020100008F0140EAF6F000EB06F74EC06F00EEC0B
:102020000CF0550E0401BD6F3D0EBE6F000EBF6F6C
:1020300045EC04F00401BD6BBE6BD0EC05F095C31C
:10204000BDF496C3BEF45F0E0401BF6F460EC06FB1
:10205000000EC16F1CEC04F00401AF6BB06B95C3B4
:10206000B1F496C3B2F4010EB36F32EC08F095C32D
:10207000BDF496C3BEF4050E0401BF6F460EC06FDB
:10208000000EC16F1CEC04F00401AF6B010EB06FC9
:1020900095C3B1F496C3B2F4010EB36F32EC08F0FD
:1020A00095C3BDF496C3BEF41C0E0401BF6F460E6B
:1020B000C06F000EC16F1CEC04F00401AF6B020E88
:1020C000B06F95C3B1F496C3B2F4010EB36F32ECA6
:1020D00008F095C3BDF496C3BEF4490E0401BF6F6A
:1020E000460EC06F000EC16F1CEC04F00401AF6B14
:1020F000030EB06F95C3B1F496C3B2F4010EB36F83
:1021000032EC08F0140E0401AF6F000EB06F74ECE7
:1021100006F06FEC0CF00EEC0CF02D0E0401BD6F10
:10212000450EBE6F000EBF6F45EC04F0EF0E0401CC
:10213000BD6F3D0EBE6F000EBF6F45EC04F08B828D
:102140000401AF6BB06B410EB16FBAEC0AF08B9229
:10215000080E0401AF6F010EB06F420EB16FBAEC02
:102160000AF0100E0401AF6F020EB06F430EB16F94
:10217000BAEC0AF0180E0401AF6F030EB06F440EF4
:10218000B16FBAEC0AF0200E0401AF6F030EB06F0E
:10219000450EB16FBAEC0AF0280E0401AF6F020EC3
:1021A000B06F460EB16FBAEC0AF0300E0401AF6F9B
:1021B000010EB06F470EB16FBAEC0AF0380E040191
:1021C000AF6FB06B480EB16FBAEC0AF0380E040175
:1021D000AF6F010EB06F490EB16FBAEC0AF0400E4E
:1021E0000401AF6F020EB06F4A0EB16FBAEC0AF085
:1021F000480E0401AF6F030EB06F4B0EB16FBAEC17
:102200000AF0500E0401AF6F030EB06F4C0EB16FA9
:10221000BAEC0AF0580E0401AF6F030EB06F4D0E0A
:10222000B16FBAEC0AF0600E0401AF6F020EB06F2E
:102230004E0EB16FBAEC0AF0680E0401AF6F010EDA
:10224000B06F4F0EB16FBAEC0AF0700E0401AF6FB1
:10225000B06B500EB16FBAEC0AF0780E0401AF6F9C
:10226000010EB06F510EB16FBAEC0AF0140E0401FA
:10227000AF6F000EB06F74EC06F00EEC0CF0FF0EBA
:102280000401BD6F3C0EBE6F000EBF6F45EC04F045
:1022900095C3BDF496C3BEF4330E0401BF6F460E62
:1022A000C06F000EC16F1CEC04F00401AF6BB06B8B
:1022B00095C3B1F496C3B2F4010EB36F32EC08F0DB
:1022C0000F0E0401AF6F000EB06F74EC06F095C3F3
:1022D000BDF496C3BEF4700E0401BF6F440EC06F10
:1022E000000EC16F1CEC04F00401AF6B020EB06F66
:1022F00095C3B1F496C3B2F4010EB36F32EC08F09B
:102300000F0E0401AF6F000EB06F74EC06F00EEC10
:102310000CF0490E0401BD6F3F0EBE6F000EBF6F83
:1023200045EC04F095C3BDF496C3BEF4C40E04019D
:10233000BF6F460EC06F000EC16F1CEC04F00401AD
:10234000AF6BB06B95C3B1F496C3B2F4020EB36F2A
:1023500032EC08F00F0E0401AF6F000EB06F74EC9A
:1023600006F01B0E0301956F040E966F95C3BDF426
:1023700096C3BEF4B30E0401BF6F460EC06F000ECD
:10238000C16F1CEC04F00401AF6B020EB06F95C37B
:10239000B1F496C3B2F4020EB36F32EC08F0140E2F
:1023A0000401AF6F000EB06F74EC06F00EEC0CF091
:1023B00095C3BDF496C3BEF4400E0401BF6F470E33
:1023C000C06F000EC16F1CEC04F0070E0401BD6F5E
:1023D000400EBE6F000EBF6F45EC04F00401AF6B02
:1023E000B06B95C3B1F496C3B2F4020EB36F32EC86
:1023F00008F0400E0401AF6F020EB06F95C3B1F448
:1024000096C3B2F4020EB36F32EC08F0140E04015E
:10241000AF6F000EB06F74EC06F00EEC0CF0060E11
:102420000401BD6F3F0EBE6F000EBF6F45EC04F0A0
:1024300095C3BDF496C3BEF4D50E0401BF6F460E1E
:10244000C06F000EC16F1CEC04F00401AF6BB06BE9
:1024500095C3B1F496C3B2F4020EB36F32EC08F038
:1024600095C3BDF496C3BEF4F50E0401BF6F460ECE
:10247000C06F000EC16F1CEC04F00401AF6B020EC4
:10248000B06F95C3B1F496C3B2F4020EB36F32ECE1
:1024900008F0140E0401AF6F000EB06F74EC06F07C
:1024A0000EEC0CF0E00E0401BD6F430EBE6F000E8B
:1024B000BF6F45EC04F01B0E0301956F040E966F81
:1024C00095C3BDF496C3BEF4860E0401BF6F470EDC
:1024D000C06F000EC16F1CEC04F00401AF6BB06B59
:1024E00095C3B1F496C3B2F4030EB36F32EC08F0A7
:1024F0001E0E0401AF6F000EB06F74EC06F00EEC10
:102500000CF095C3BDF496C3BEF4750E0401BF6F05
:10251000460EC06F000EC16F1CEC04F00401AF6BDF
:10252000B06B95C3B1F496C3B2F4010EB36F32EC45
:1025300008F0900E0401BD6F440EBE6F000EBF6F19
:1025400045EC04F00401AF6B020EB06FB16B58ECB8
:102550000AF0140EAF6F020EB06F010EB16F58EC9F
:102560000AF0280EAF6F020EB06F020EB16F58EC7A
:102570000AF03C0EAF6F020EB06F030EB16F58EC55
:102580000AF0460EAF6F020EB06F430EB16FBAEC99
:102590000AF0600E0401AF6F020EB06F7C0EB16FD7
:1025A000BAEC0AF0680E0401AF6F020EB06F430E72
:1025B000B16FBAEC0AF0140E0401AF6F000EB06FE9
:1025C00074EC06F00EEC0CF0450E0401BD6F400EED
:1025D000BE6F000EBF6F45EC04F095C3BDF496C30B
:1025E000BEF4690E0401BF6F470EC06F000EC16FCD
:1025F0001CEC04F00301976B986B800E9819006E29
:10260000800E005C02E1070E975D13E2040E006E7F
:1026100097C3BDF4005005E00401BD37BD91FF0F25
:10262000FAD797C3BEF481EC04F00301974B982BC3
:10263000E4D7140E0401AF6F000EB06F74EC06F017
:102640000EEC0CF0EF0E0401BD6F440EBE6F000ED9
:10265000BF6F45EC04F00301976B986B0401BD6BF1
:102660000B0EBE6F81EC04F0100E03019725006E77
:10267000000E9821016E00C097F301C098F300C0CE
:10268000BDF4020E0401BE6F81EC04F0100E0301D4
:102690009725006E000E9821016E00C097F301C0CF
:1026A00098F300C0BDF4010E0401BE6F81EC04F08C
:1026B000100E03019725006E000E9821016E00C0D8
:1026C00097F301C098F300C0BDF40A0E0401BE6F79
:1026D00081EC04F0100E03019725006E000E982186
:1026E000016E00C097F301C098F300C0BDF4090E5D
:1026F0000401BE6F81EC04F0140E03019725006EF7
:10270000000E9821016E00C097F301C098F300C03D
:10271000AFF4010E0401B06F030EB16F58EC0AF074
:10272000100E03019725006E000E9821016E00C067
:1027300097F301C098F300C0AFF4010E0401B06F2D
:10274000430EB16FBAEC0AF08978140E0401AF6F32
:10275000000EB06F74EC06F00EEC0CF02B0E0401C2
:10276000BD6F440EBE6F000EBF6F45EC04F0040158
:10277000AF6BB06B800EB16F040EB26F6C0EB36FA7
:10278000350EB46F000EB56F43EC0EF00F0EAF6F49
:10279000000EB06F74EC06F00EEC0CF04C0E040161
:1027A000BD6F450EBE6F000EBF6F45EC04F0040117
:1027B000AF6BB06B800EB16F040EB26F6C0EB36F67
:1027C000390EB46F000EB56F43EC0EF00F0EAF6F05
:1027D000000EB06F74EC06F00EEC0CF06A0E040103
:1027E000BD6F450EBE6F000EBF6F45EC04F00401D7
:1027F000AF6BB06B800EB16F040EB26F6C0EB36F27
:10280000370EB46F000EB56F43EC0EF00F0EAF6FC6
:10281000000EB06F74EC06F00EEC0CF0D50E040157
:10282000BD6F450EBE6F000EBF6F45EC04F06FEC40
:102830000CF00301976B986B800E9819006E800E58
:10284000005C02E17F0E975D17E297C3D2F4250E7C
:102850009725E96E000E9821EA6EE9CFE9FFEACFED
:10286000EAFFEECFD3F4010E0401D46F18EC02F0AE
:102870000301974B982BE0D7F6EC0CF0140E0401F3
:10288000AF6F000EB06F74EC06F00E0E0401BD6F5A
:10289000450EBE6F000EBF6F45EC04F00EEC0CF061
:1028A0006FEC0CF095C3BDF496C3BEF48B0E04011F
:1028B000BF6F460EC06F000EC16F1CEC04F0040128
:1028C000AF6B010EB06F95C3B1F496C3B2F4010EB5
:1028D000B36F32EC08F0020E0401D26F020ED36F18
:1028E000010ED46F18EC02F07D0E0401D26FD36B91
:1028F000010ED46F18EC02F0020E0401D26F1D0E0F
:10290000D36F010ED46F18EC02F07D0E0401D26F6C
:102910001D0ED36F010ED46F18EC02F0F6EC0CF024
:10292000140E0401AF6F000EB06F74EC06F0B20E1F
:102930000401BD6F400EBE6F000EBF6F45EC04F08A
:102940000EEC0CF06FEC0CF00301976B986B800EA3
:102950009819006E800E005C02E17F0E975D16E212
:1029600097C3D2F4060E0401D36F010ED46F18EC96
:1029700002F097C3D2F4160E0401D36F010ED46F88
:1029800018EC02F00301974B982BE1D7F6EC0CF012
:10299000140E0401AF6F000EB06F74EC06F00EEC75
:1029A0000CF06FEC0CF0870E0401BD6F450EBE6F8E
:1029B000000EBF6F45EC04F0010E0401BD6F010E67
:1029C000BE6F7E0EBF6F1F0EC06F010EC16FE1ECB8
:1029D00002F0010EBD6F1F0EBE6F7E0EBF6F010EA7
:1029E000C06F010EC16FE1EC02F0F6EC0CF0140EBA
:1029F0000401AF6F000EB06F74EC06F0B50E040169
:102A0000BD6F430EBE6F000EBF6F45EC04F00EECC1
:102A10000CF06FEC0CF00301976B986B800E98191B
:102A2000006E800E005C02E10F0E975D2BE2975165
:102A3000010F006E00C0AFF400C0B0F497517E08E3
:102A40000401B16F030197511F080401B26FB36B0A
:102A5000010EB46F8AEC0CF0F6EC0CF00B0E0B6E62
:102A6000260E0C6E5D0E0D6E0D2EFED70C2EFCD7B5
:102A70000B2EFAD700000000030E03019727000E6B
:102A80009823CCD7190E0401AF6F000EB06F74EC11
:102A900006F0890E0401BD6F430EBE6F000EBF6FBE
:102AA00045EC04F00EEC0CF06FEC0CF00C0E030196
:102AB000976F000E986F800E006E800E9819005C64
:102AC00002E1975102082CE29751010F006E00C0FD
:102AD000AFF400C0B0F497517E080401B16F030158
:102AE00097511F080401B26F010EB36F010EB46F4E
:102AF0008AEC0CF0F6EC0CF00B0E0B6E260E0C6E46
:102B00005D0E0D6E0D2EFED70C2EFCD70B2EFAD7B8
:102B100000000000020E0301975F000E985BCBD708
:102B20001E0E0401AF6F000EB06F74EC06F00EECD9
:102B30000CF0D00E0401BD6F440EBE6F000EBF6FCF
:102B400045EC04F06FEC0CF095C3BDF496C3BEF4F5
:102B5000510E0401BF6F470EC06F000EC16F1CEC19
:102B600004F00401AF6BB06B95C3B1F496C3B2F43B
:102B7000010EB36F32EC08F095C3BDF496C3BEF4FA
:102B80008C0E0401BF6F470EC06F000EC16F1CECAE
:102B900004F00401AF6B010EB06F95C3B1F496C39E
:102BA000B2F4010EB36F32EC08F0040E0301976F1C
:102BB000000E986F800E9819006E800E005C02E186
:102BC000110E975D22E2400E0401AF6F0F0EB06F41
:102BD00097C3B1F4B26B010EB36F4FEC0DF0F6EC8E
:102BE0000CF00B0E0B6E260E0C6E5D0E0D6E0D2E88
:102BF000FED70C2EFCD70B2EFAD700000000020ED9
:102C000003019727000E9823D5D71E0E0401AF6F3E
:102C1000000EB06F74EC06F00EEC0CF0B00E040178
:102C2000BD6F440EBE6F000EBF6F45EC04F06FEC3D
:102C30000CF095C3BDF496C3BEF4490E0401BF6FFA
:102C4000470EC06F000EC16F1CEC04F00401AF6BA7
:102C5000010EB06F95C3B1F496C3B2F4010EB36F19
:102C600032EC08F095C3BDF496C3BEF4710E0401B6
:102C7000BF6F470EC06F000EC16F1CEC04F0040163
:102C8000AF6B010EB06F95C3B1F496C3B2F4010EF1
:102C9000B36F32EC08F0040E0301976F000E986FCB
:102CA000800E9819006E800E005C02E1110E975D97
:102CB00034E2400E0401AF6F0F0EB06F97C3B1F452
:102CC000010EB26F010EB36F4FEC0DF0F6EC0CF08D
:102CD0000B0E0B6E260E0C6E5D0E0D6E0D2EFED7BE
:102CE0000C2EFCD70B2EFAD700000000400E04017A
:102CF000AF6F0F0EB06F020E0301975D0401B16F4D
:102D0000010EB26FB36B4FEC0DF0F6EC0CF0020E4F
:102D100003019727000E9823C3D71E0E0401AF6F3F
:102D2000000EB06F74EC06F06FEC0CF0F6EC0CF0EB
:102D3000040E0401BD6F470EBE6F000EBF6F45EC61
:102D400004F089EF10F0FFD7000000000000000041
:102D50000000000000000000000000F8000000007B
:102D6000000000333000000000100C06100C0600BC
:102D7000000000000000000040C07840C078400023
:102D8000043F04043F040400007088FC0830000085
:102D9000001820FF211E0000F008F000E0180000DD
:102DA00000211C031E211E0000F008887000000096
:102DB0001E2123241927211010160E0000000000E8
:102DC0000000000000000000000000E01804020005
:102DD000000000071820400000020418E000000076
:102DE0000040201807000000404080F08040400074
:102DF0000202010F01020200000000F000000000CA
:102E00000101011F0101010000000000000000009D
:102E100080B0700000000000000000000000000012
:102E2000000101010101010100000000000000009B
:102E30000030300000000000000000008060180436
:102E4000006018060100000000E010080810E00013
:102E5000000F102020100F00001010F800000000DC
:102E60000020203F20200000007008080888700023
:102E700000302824222130000030088888483000A3
:102E80000018202020110E000000C02010F80000C3
:102E900000070424243F240000F80888880808005C
:102EA0000019212020110E0000E010888818000071
:102EB000000F112020110E0000380808C838080043
:102EC0000000003F000000000070880808887000C3
:102ED000001C222121221C0000E010080810E00044
:102EE0000000312222110F00000000C0C0000000CD
:102EF00000000030300000000000008000000000F2
:102F000000008060000000000000804020100800E9
:102F100000010204081020004040404040404000B2
:102F2000040404040404040000081020408000008D
:102F30000020100804020100007048080808F00092
:102F40000000003036010000C030C828E810E00062
:102F50000718272423140B000000C038E0000000ED
:102F6000203C23020227382008F888888870000057
:102F7000203F202020110E00C0300808080838002B
:102F8000071820202010080008F808080810E000A2
:102F9000203F202020100F0008F88888E808100043
:102FA000203F20202320180008F88888E808100017
:102FB000203F200003000000C0300808083800004F
:102FC00007182020221E020008F808000008F80850
:102FD000203F210101213F20000808F808080000D7
:102FE0000020203F2020000000000808F80808000A
:102FF000C08080807F00000008F888C02818080082
:10300000203F20012638200008F8080000000000BA
:10301000203F20202020300008F8F800F8F80800B1
:10302000203F003F003F200008F830C00008F808AB
:10303000203F200007183F00E01008080810E000BB
:103040000F10202020100F0008F808080808F000D2
:10305000203F210101010000E01008080810E000F5
:103060000F18242438504F0008F88888888870008A
:10307000203F2000030C302000708808080838002A
:103080000038202121221C00180808F80808180020
:103090000000203F2000000008F808000008F808A1
:1030A000001F202020201F000878880000C8380852
:1030B000000007380E010000F80800F80008F800CA
:1030C000033C0700073C0300081868808068180864
:1030D00020302C03032C30200838C800C8380800E2
:1030E0000000203F2000000010080808C838080031
:1030F0002038262120201800000000FE02020200D5
:103100000000007F40404000000C30C00000000084
:10311000000000010638C00000020202FE000000AC
:10312000004040407F000000000004020202040052
:10313000000000000000000000000000000000008F
:103140008080808080808080000202040000000077
:10315000000000000000000000008080808000006F
:103160000019242222223F2008F80080800000005D
:10317000003F112020110E00000000808080000020
:10318000000E112020201100000000808088F8002F
:10319000000E112020103F20000080808080000061
:1031A000001F222222221300008080F088888818C5
:1031B0000020203F202000000000808080808000D0
:1031C000006B94949493600008F800808080000065
:1031D000203F210000203F20008098980000000040
:1031E0000020203F20200000000000809898000070
:1031F00000C08080807F000008F800008080800090
:10320000203F24022D302000000808F800000000B4
:103210000020203F2020000080808080808080006F
:10322000203F20003F20003F808000808080000001
:10323000203F210000203F2000008080808000008F
:10324000001F202020201F008080008080000000C0
:1032500080FFA12020110E000000008080808000EF
:10326000000E112020A0FF808080800080808000E0
:1032700020203F212000010000008080808080000D
:103280000033242424241900008080E08080000082
:103290000000001F202000008080000000808000CF
:1032A000001F202020103F20808080000080808030
:1032B00000010E30080601008080008000808080C0
:1032C0000F300C030C300F000080800080808000E5
:1032D0000020312E0E312000808080000080808010
:1032E00080818E70180601000080808080808000C0
:1032F0000021302C2221300000000000807C0202DE
:1033000000000000003F404000000000FF000000FF
:1033100000000000FF0000000002027C80000000AE
:103320000040403F000000000006010102020404CA
:10333000000000000000000000000000000000008D
:10334000002F000000000700070000147F147F1406
:1033500000242A7F2A12006264081323003649558C
:10336000225000000503000000001C224100000064
:1033700041221C000014083E08140008083E0808FA
:10338000000000A060000008080808080000606055
:103390000000002010080402003E5149453E000094
:1033A000427F4000004261514946002141454B3176
:1033B000001814127F10002745454539003C4A4942
:1033C00049300001710905030036494949360006B4
:1033D0004949291E0000363600000000563600001C
:1033E0000008142241000014141414140000412297
:1033F000140800020151090600324959513E007C6F
:103400001211127C007F49494936003E4141412258
:10341000007F4141221C007F49494941007F090941
:103420000901003E4149497A007F0808087F0000F1
:10343000417F4100002040413F01007F08142241AC
:10344000007F40404040007F020C027F007F040864
:10345000107F003E4141413E007F09090906003EC0
:103460004151215E007F09192946004649494931E9
:103470000001017F0101003F4040403F001F20400C
:10348000201F003F4038403F0063140814630007CA
:103490000870080700615149454300007F41410021
:1034A000000204081020000041417F0000040201D6
:1034B000020400404040404000000102040000209F
:1034C00054545478007F48444438003844444420DD
:1034D00000384444487F00385454541800087E098A
:1034E00001020018A4A4A47C007F08040478000052
:1034F000447D4000004080847D00007F102844000F
:103500000000417F4000007C04180478007C08041F
:10351000047800384444443800FC2424241800185B
:10352000242418FC007C0804040800485454542047
:1035300000043F444020003C4040207C001C2040D0
:10354000201C003C4030403C004428102844001C13
:10355000A0A0A07C004464544C441414141414140B
:103560000F090F090000000000000000000305091A
:1035700011FF118905C300E000F000F80000000011
:103580000000004428FF11AA4400000000000000D1
:10359000000000000000000000000000000000002B
:1035A000000000000000000000000000000000001B
:1035B000000000000000000000000000000000000B
:1035C000000000000000830138448292927401835D
:1035D000000000000000007C44C7017D7D7D7D016E
:1035E0007D7D7D7D017D7D7D7D01FF0000000000F2
:1035F00000010001000100010001000100000000C5
:1036000000000000000101000000000000000000B8
:1036100000000000000000000000000000000000AA
:10362000000000000000000000000000000000009A
:10363000000000000000000000000000000000008A
:103640000000000000000101000000000000010176
:103650000000000000000000000101010101010163
:10366000010101010101010101010100000000004F
:103670000000000000404040404000006D6D6D6D56
:103680006D000060606060600000404040404000AD
:10369000000000000000000000000000000000002A
:1036A000000000000000000000000000000000001A
:1036B000000000000000000000000000000000000A
:1036C00000000000000000000000000000000000FA
:1036D00000000000000000000000000000000000EA
:1036E00000000000000000000000000000000000DA
:1036F0000000000000DBDBDBDBDB0000DBDBDBDB17
:10370000DB0000DBDBDBDBDB0000DBDBDBDBDB0050
:1037100000DADADADADA0000D8D8D8D8D80000C06F
:10372000C0C0C0C00000C0C0C0C0C00000C0C0C099
:10373000C0C00000C0C0C0C0C000008080808080C9
:103740000000000000000000000000000000000079
:103750000000000000000000000000000000000069
:103760000000000000000000000000000000000059
:103770000000000000000000000000000000000049
:103780000000000000000000000000000000000039
:103790000000000000000000000000000000000029
:1037A0000000000000000000000000808080000099
:1037B000000000000000000000000000008080C049
:1037C000C000000000000000000000000000000039
:1037D00000000000000000000000000000000000E9
:1037E00000000000000000000000000000000000D9
:1037F00000000000000000000000000000000000C9
:1038000080C0E0F0F8FCF8E00000000000000000DC
:1038100000000000000000000080808080800080A8
:103820008000000000808080808000FFFFFF00009B
:1038300000008080808000008080000080FFFF808A
:1038400080008080008080808000808000000000F8
:1038500000808000008C8E84000080F8F8F88000E2
:10386000000000000000000000000000F0F0F0F098
:10387000F0F0F0F0F0F0F0F0E0E0C08000E0FCFEEE
:10388000FFFFFF7FFFFFFFFFFF00000000000000C1
:1038900000000000000000FEFFC70101010183FFDE
:1038A000FF00007CFEC70101010183FFFFFF00381C
:1038B000FEC78301010183C7FFFF000001FFFF0175
:1038C0000100FFFF0701010100007FFF80000000F1
:1038D000FFFF7F0000FFFFFF000001FFFFFF01006F
:1038E000000000000000000000000000030F3F7F08
:1038F0007FFFFFFFFFFFFFFFE7C7C78F8F9FBFFF60
:10390000FFC3C0F0FFFFFFFFFFFCFCFCFCFCFCFC66
:10391000FCF8F8F0F0E0C000010303030303010327
:103920000300000000010303030301010301000081
:10393000000103030303010103030000000303006C
:103940000000030300000000000000010303030364
:103950000301000000010301000000030301000057
:103960000000000000000000000000000000000057
:1039700000F0F8F8F878787878F8F0E0E080000067
:103980000000000000000000000000000000000037
:10399000000000000000000000000000000000F037
:1039A000F0F8F000000000F8F8F8F8787878787807
:1039B0007878787070100000000000F0F0F0F000EF
:1039C00000000000000000000000000000000000F7
:1039D0000000000000F0F0F0F00000000000000027
:1039E00000000000000000000000000000000000D7
:1039F000FFFFFFFFF0F0F0F0F87F1F1F0F00000047
:103A000080F0F8F87E1E1E1EFEF8F8F80000000098
:103A1000F8F8F8F800000000F8F8F8F80000FFFFE8
:103A2000FFFF00000000FFFFFFFF787878787878CC
:103A300078781010000000000000F8F8F8F8000096
:103A40000000F8F8F8F800000000F8F8F8F80000B6
:103A500000000000F8FEF8F800008080F0F87E7E9C
:103A60001E1E7E7EFEF8E0E000000000000000FF69
:103A7000FFFFFF0000000000000000000000001F2A
:103A8000FFFFFFE0E0E0E0FFFFFFFFE00000007F5E
:103A9000FFFFFFE0E0E0E0FFFFFFFF0000FFFFFFB0
:103AA000FF00000000FFFFFFFF000000000000001B
:103AB0000000000000000000000707FFFFF8F8000A
:103AC000007F7FFFFFE0E0E0E0FFFFFFFF0000007E
:103AD00000000007FFFFFFF8001F1FFFFFF0F0E0EE
:103AE000E0F0F0FF7F1F1F00000000000000000159
:103AF00000000000000000000000000000000000C6
:103B000001010101010100000101010000000000AC
:103B1000010101010101010101010000000001009A
:103B20000000000000000100000000000000000094
:103B30000000000F1F1F7EF8F0F0FF7F1F1F000026
:103B40000000000101010101010101010F0F1F7EB1
:103B5000F8F8F0FF7F7F1F00000000000101010165
:103B600001010000000000006147007847007F4726
:103B7000005947000F11131517191A1B1C1D1E1E83
:103B80001E1E1D1C1B1918161412100E0C0A0806F6
:103B90000503020100000000010203040507090BF0
:103BA0000D0F11131517191A1B1C1D1E1E1E1E1D8D
:103BB0001C1B1918161412100E0C0A080605030215
:103BC0000100000000010203040507090B0D0F119D
:103BD000131517191A1B1C1D1E1E1E1E1D1C1B193A
:103BE00018161412100E0C0A080605030201000034
:103BF0000000010200000000694200794100A94173
:103C000000D94100194100494100294300F942000F
:103C1000594300C94200394200094200994200A2BA
:103C20004500A63D007D3E00A93C00C93F00373E4F
:103C300000E54600BC45003D3C0006000020417503
:103C400074726573203A2020424D505F696D616740
:103C500065735F3132387833325F323032312E69FA
:103C60006E63200D0A204F4C45445F313238783363
:103C7000325F493243315F323032315F30322E634E
:103C8000206574202A2E680D0A204F4C45445F3170
:103C900032387833325F5461626C65735F32303230
:103CA000315F30322E680D0A0020536F75726365E4
:103CB000203A2020544553545F4D696E695F4F4C44
:103CC00045445F535344313330365F3132387833B3
:103CD000325F776974685F493243315F48575F4D9F
:103CE000696B726F435F31384632364B32325F5FF9
:103CF000323032345F313230382E63200D0A0020EA
:103D000041666669636865205465787465206465FA
:103D1000203231206361727320706172206C696798
:103D20006E6520285461696C6C65206D696E693D13
:103D3000203129203A0D0A20414243444546474854
:103D4000494A4B4C4D4E4F5051525354555657586B
:103D5000595A0D0A002041666669636865205465FA
:103D6000787465206465203231206361727320703D
:103D70006172206C69676E6520285461696C6C659E
:103D8000206D696E693D203129203A0D0A2041429B
:103D9000434445464748494A4B4C4D4E4F5051527B
:103DA0005354550D0A00204469726563746F72792B
:103DB000203A20433A5C5F4D696B726F435C5F3120
:103DC000384632364B32325F546573745F4D696EDC
:103DD000695F4F4C45445F4932435F323078313040
:103DE0006D6D5F4932435F32303234200D0A00205E
:103DF00057726974655F436861725F417428582027
:103E0000656E20706978656C20283020E0203132A2
:103E100037292C206C69676E65205920283020E0F6
:103E20002033292C636F64652061736369692063A3
:103E3000686172290D0A0020493243312048572019
:103E400061766563204D696B726F43204C696272C5
:103E5000617279202C5465726D696E616C20706F8F
:103E60007572206465627567206574205669737584
:103E70002070726F6772616D6D650D0A002050725F
:103E80006F6A6574203A20204D696E695F4F4C451A
:103E9000445F3132387833325F32357831306D6D8E
:103EA0005F493243315F48575F4D435F3138463297
:103EB000364B32325F323032342E6D637070690DA2
:103EC0000A00205465737420636F6E736F6D6D61AB
:103ED00074696F6E206475204C4344204F4C4544F8
:103EE00020416C6C756DE92031303025204F4E201B
:103EF000202831332E366D4120736F757320332E99
:103F00003356290D0A00204166666963686167655A
:103F100020285461696C6C65203229206465203A40
:103F20002048454C4C4F20467269656E64732C20C6
:103F3000486F772061726520796F75203F2E206170
:103F40007420783D30200D0A002041666669636860
:103F500065203136206361727320285461696C6C6E
:103F6000653D203229203A30313233343536373806
:103F70003930313233343520617420783D302C2093
:103F80006C69676E652032200D0A002054657374D9
:103F900020636F6E736F6D6D6174696F6E206475F1
:103FA00020204C4344204F4C454420204554454953
:103FB0004E542028312E35336D4120736F75732098
:103FC000332E335629200D0A0020444556494345D7
:103FD000203A20204D696E69204F4C4544204449C9
:103FE00053504C4159204949432049324320302EF7
:103FF000393120203132387833322020323578314F
:10400000306D6D200D0A0020416666696368652089
:1040100038206361727320285461696C6C653D209F
:1040200032293A203031323334353637206174202A
:10403000783D302C36342C206C69676E6520302C2E
:1040400032200D0A00204269675F61666669636815
:104050006167652820756E7369676E6564206368A3
:10406000617220706F73582C20756E7369676E656E
:10407000642063686172204E20290D0A00204F4C95
:10408000454420535344313330362031323878336D
:1040900032204932432C2020696E697469616C6951
:1040A00073E92028656E206D6F6465203229200D2C
:1040B0000A00204472617720486F72697A2E4C6939
:1040C0006E65207769746820447261775F50697803
:1040D000656C202061742020793D3620657420793C
:1040E0003D32320D0A00205465737420696E746588
:1040F00072727570742054696D657231202032308F
:10410000207820313030206D73656320736F6974BF
:104110002032736563200D0A000000000000C0E03B
:10412000F8FCFFFFFFFFFF0000C0E0F8FCFFBF8FBF
:104130008381FFFFFFFFFF8080070707070707074F
:104140000707FFFFFFFFFF0707000080FCFFFFFFDF
:104150003F1F1F1F1F1F1F1F0000183F3F3F3F1F14
:104160000F0F0F1FFFFEFEF8E000061F3F7F7FFCD2
:10417000F0F0F0F87F7F3F1F07000000C0E0E0F0A4
:10418000F87CFEFFFFFFFF000000000003010100BC
:104190000000FFFFFFFFFF00000000000000000024
:1041A0000000FFFFFFFFFF000000E0F8FCFEFE1F25
:1041B0000F0F0F1FFFFEFEFCF0000000000080C08C
:1041C000E0F0F8FE7F3F1F070100C0F8FCFFFFFF93
:1041D000FFF9F9F8F8F8F8F8F80030787E7E7F1FDC
:1041E0000F0F1FFFFEFEFCF00000000000000000AB
:1041F0000E0E0F1FFBFBF9F0C000061F3F7F7FFC78
:10420000F0F0F0FC7F7F3F1F07000000000000007F
:10421000000000000000000000000000000000009E
:10422000000000000000000000000000000000008E
:10423000000000000000000000000000000000007E
:10424000000000000000000000000000000000006E
:10425000000000000000000000000000000000005E
:10426000000000FFFFFFFF00000080F0FCFEFE3FAB
:104270000F0F0F3FFEFEFCF08000FFFFFFFFFF006F
:1042800000000000FFFFFFFFFF00030F3F7F7FFCE8
:10429000F0F0F0FC7F7F3F0F01000000001FE00006
:1042A00000000018C00000000018C0000000001F3F
:1042B000C00000000000000000000000000000003E
:1042C00000000000000000000000E0F8FCFEFF1FFE
:1042D0000F0F0F1FFEFEFCF08000070F3F3F7F7C9B
:1042E0007878783CFFFFFFFFFF000E3E7E7EFEF8F1
:1042F000F0F0F07C7F3F1F0F01001F1F1F1F1F1FCB
:104300001F1F9FFFFFFF3F1F0F0000000000E0F88E
:10431000FCFF7F0F0300000000000000F0FFFFFF24
:10432000FF07000000000000000080F0F8FCFE3EE7
:104330000F0F0F1F7F7E7E7C7000FFFFFFFFFF3C93
:104340001E1E1E3EFEFCFCF0E000010F3F7F7FF8CA
:10435000F0F0F0F8FF7F3F1F0700F0FCFEFEFF1FAC
:104360000F0F0F1FFFFEFEFCF00081C3E7FFFF7E73
:104370003C3C3C7EFFFFE7C381000F3F7F7FFFF89F
:10438000F0F0F0F8FF7F7F3F0F20447261772072DA
:10439000656374616E676C65732028506C65696E27
:1043A00073292061742020312C312C3132362C338A
:1043B00030200D0A002044726177207265637461B9
:1043C0006E676C6573202876696465732920617453
:1043D0002020312C312C3132362C3330200D0A0084
:1043E0002041666669636861676520287461696C4D
:1043F0006C65203D203329206465203A2031392E18
:1044000038B0430D0A0020496E697420496E746506
:1044100072727570742054696D6572312020262087
:1044200055415254205258200D0A002041666669B9
:10443000636861676520496D6167652050726F76BA
:1044400069646572205250432031200D0A00202EED
:104450002E2E2057616974696E67204B6579626FF3
:1044600061726420546F75636820666F72203C002F
:104470004142434445464748494A4B4C4D4E4F50B4
:104480005152535455565758595A2E2E657463003D
:1044900020577269746520342063617261637465AA
:1044A000726573207370656369617578200D0A0009
:1044B000204472617720436572636C657320506C91
:1044C00065696E732063656E7472E973200D0A006E
:1044D000204472617720436572636C65732076694E
:1044E0006465732063656E7472E973200D0A0020A1
:1044F000416666696368616765204D697874652007
:104500006465203A2032312E39B0430D0A00204430
:1045100072617720506978656C7320617420203156
:104520002C312C3132362C3330200D0A00204166DC
:104530006669636865206C657474726573204120D8
:10454000422043202E2E2E51200D0A002041666667
:1045500069636861676520496D6167652070617591
:104560006C666A756A6F200D0A0020416666696391
:104570006861676520496D616765204164616672A5
:10458000756974200D0A00204F4C45445F4C696EDC
:10459000657320646961676F6E616C657320200DBF
:1045A0000A00204D696B726F6320372E362E302043
:1045B00031384632364B3232200D0A0020464F53F6
:1045C000433D2020496E7465726E65203136204D62
:1045D000487A0D0A00204166666963686167652054
:1045E00073696E75736F696465200D0A000D0A208A
:1045F00044657669636520617420616472657373D4
:1046000065203A20004F4C45442053697A6520319B
:104610003238783332203235783130004932432015
:1046200048617264204D432030322F30322F3230B7
:10463000323100416666696368652032312063610A
:10464000722E73697A653D31002A202A202A202A99
:10465000202A202A202A202A202A202A202A002A2A
:10466000202A202A202A202A202A202A202A202AFA
:10467000202A202A005772697465203420636172F1
:104680002E73706563696175782000506978656C78
:104690007320617420322C322C3132352C323900A7
:1046A0002050726573656E746174696F6E203A2074
:1046B0000D0A003031323334353637383930313243
:1046C000333435004166662E3136206368722073BC
:1046D000697A6532002048454C4C4F204672696526
:1046E0006E6473200020416C696D203D20332E36AE
:1046F00020560D0A0020486F772061726520796F7F
:1047000075203F000D0A204E6578742E2E200D0A6C
:1047100000204932433120696E69740D0A00204F30
:104720004C454420434C53200D0A0020666F756EA3
:1047300064204F4B0D0A0020536563203E0D0A0094
:10474000303132333435363700436572636C65730C
:1047500000436572636C6573000F090F0000000071
:104760000000007E66667E0000303132333435361C
:1047700000706C65696E7300C030383E383060067A
:104780000C1C7C1C0C0631392E38320056696465CD
:104790007300474F0D0A00FF10EE19F0D50E006EA2
:1047A000010E016E680EF66E3B0EF76E000EF86E8F
:1047B0006CEC06F01200FFFFFFFFFFFFFFFFFFFFA3
:020000040030CA
:0D00010028183CFFBF81FF0FC00FE00F402B
:00000001FF
